:1003680090E668E0FF74FFF0E0B40B04EFF0D322EE
:0603780090E668EFF0C3FF
:01037E00225C
:1001B500907FE9E064A360030202C5A3E07508002F
:1001C500F509A3E0FEE4EE4208907FEEE0750A0033
:1001D500F50BA3E0FEE4EE420A907FE8E064407090
:1001E50064E50B450A70030202D6E4907FC5F090E2
:1001F5007FB4E020E3F9907FC5E0750C00F50DE4D0
:10020500FCFDC3ED950DEC950C501F74C02DF582CA
:10021500E4347EF583E0FFE5092DF582E5083CF53C
:1002250083EFF00DBD00010C80D8E50D2509F5091A
:10023500E50C3508F508C3E50B950DF50BE50A95B5
:100245000CF50A809C907FE8E064C060030202D64A
:10025500E50B450A607BC3E50B9440E50A94005025
:1002650008850A0C850B0D8006750C00750D40E49C
:10027500FCFDC3ED950DEC950C501FE5092DF582A0
:10028500E5083CF583E0FF74002DF582E4347FF545
:1002950083EFF00DBD00010C80D8907FB5E50DF022
:1002A5002509F509E50C3508F508C3E50B950DF5A8
:1002B5000BE50A950CF50A907FB4E030E29280F7E1
:1002C500907FE9E0B4AC0AE4907F00F0907FB5043C
:0802D500F0907FB4E04402F058
:0102DD0022FE
:1000800090E6B9E064A36003020198A3E07508005C
:10009000F509A3E0FEE4EE420890E6BEE0750A0032
:1000A000F50BA3E0FEE4EE420A90E6B8E06440708F
:1000B00066E50B450A70030201ADE490E68AF0A301
:1000C000F090E6A0E020E1F990E68BE0750C00F5F9
:1000D0000DE4FCFDC3ED950DEC950C501F74402D07
:1000E000F582E434E7F583E0FFE5092DF582E508C4
:1000F0003CF583EFF00DBD00010C80D8E50D25091E
:10010000F509E50C3508F508C3E50B950DF50BE58C
:100110000A950CF50A809A90E6B8E064C060030284
:1001200001ADE50B450A70030201ADC3E50B944038
:10013000E50A94005008850A0C850B0D8006750CA5
:1001400000750D40E4FCFDC3ED950DEC950C501FC2
:10015000E5092DF582E5083CF583E0FF74402DF5B7
:1001600082E434E7F583EFF00DBD00010C80D8E4A4
:1001700090E68AF0A3E50DF02509F509E50C3508B0
:10018000F508C3E50B950DF50BE50A950CF50A90FE
:10019000E6A0E030E18C80F790E6B9E0B4AC0E90D8
:1001A000E7407401F0E490E68AF0A304F090E6A042
:0401B000E04480F0B7
:0101B4002228
:1002DE00C2011203689200907F95E044C0F0D2E80C
:1002EE0030000890E65D74FFF08006907FAB74FFDF
:1002FE00F030000890E6687408F08007907FAFE059
:10030E004401F030000890E65C7401F08006907FA6
:10031E00AE7401F0D2AF3001FD30000512008080C6
:08032E00031201B5C20180EECB
:03000300020336BF
:10033600C0E0C083C082C085C084C086758600D2F6
:10034600015391EF30000890E65D7401F08006904D
:100356007FAB7401F0D086D084D085D082D083D094
:02036600E03283
:03004300020400B4
:0404000002033600BD
:0300000002037F79
:0C037F00787FE4F6D8FD7581200202DED4
:00000001FF
